
 MMSYSTEM

 Start     Length     Name                   Class
 0001:0000 0073BH     FIX                    CODE
 0002:0000 007FEH     INIT                   CODE
 0003:0000 01506H     WAVE                   CODE
 0004:0000 008EDH     _TEXT                  CODE
 0005:0000 03F50H     MCI                    CODE
 0006:0000 00A12H     MIDI                   CODE
 0007:0000 018ACH     MMIO                   CODE
 0008:0000 006CFH     RARE                   CODE
 0009:0000 013E4H     MIXER                  CODE
 000A:0000 0001AH     INTDS                  DATA
 000B:0000 000A4H     _DATA                  DATA
 000B:00A4 00012H     CONST                  CONST
 000B:00B6 00020H     _BSS                   BSS
 000B:00E0 00166H     c_common               BSS

 Origin   Group
 000B:0   DGROUP

 Address   Export                  Alias

 0008:058C AUXGETDEVCAPS           AUXGETDEVCAPS
 0008:0572 AUXGETNUMDEVS           AUXGETNUMDEVS
 0008:05D4 AUXGETVOLUME            AUXGETVOLUME
 0008:0632 AUXOUTMESSAGE           AUXOUTMESSAGE
 0008:0610 AUXSETVOLUME            AUXSETVOLUME
 0001:049E DRIVERCALLBACK          DRIVERCALLBACK
 0004:0036 DRIVERPROC              DRIVERPROC
 0004:059B DRVCLOSE                DRVCLOSE
 0004:05AA DRVDEFDRIVERPROC        DRVDEFDRIVERPROC
 0004:05A0 DRVGETMODULEHANDLE      DRVGETMODULEHANDLE
 0004:0596 DRVOPEN                 DRVOPEN
 0004:05A5 DRVSENDMESSAGE          DRVSENDMESSAGE
 0008:0022 JOYGETDEVCAPS           JOYGETDEVCAPS
 0008:008C JOYGETNUMDEVS           JOYGETNUMDEVS
 0008:00A8 JOYGETPOS               JOYGETPOS
 0008:0112 JOYGETTHRESHOLD         JOYGETTHRESHOLD
 0008:0176 JOYRELEASECAPTURE       JOYRELEASECAPTURE
 0008:0318 JOYSETCALIBRATION       JOYSETCALIBRATION
 0008:01DE JOYSETCAPTURE           JOYSETCAPTURE
 0008:02CE JOYSETTHRESHOLD         JOYSETTHRESHOLD
 0001:02E3 MCIDRIVERNOTIFY         MCIDRIVERNOTIFY
 0005:2DC6 MCIDRIVERYIELD          MCIDRIVERYIELD
 0005:146C MCIEXECUTE              MCIEXECUTE
 0005:3348 MCIFREECOMMANDRESOURCE  MCIFREECOMMANDRESOURCE
 0005:1906 MCIGETCREATORTASK       MCIGETCREATORTASK
 0005:188A MCIGETDEVICEID          MCIGETDEVICEID
 0005:1718 MCIGETDEVICEIDFROMELEMENTID  MCIGETDEVICEIDFROMELEMENTID
 0005:2D1E MCIGETDRIVERDATA        MCIGETDRIVERDATA
 0005:155A MCIGETERRORSTRING       MCIGETERRORSTRING
 0005:2EAA MCIGETYIELDPROC         MCIGETYIELDPROC
 0005:30CA MCILOADCOMMANDRESOURCE  MCILOADCOMMANDRESOURCE
 0005:3D52 MCIPARSECOMMAND         MCIPARSECOMMAND
 0005:04E6 MCISENDCOMMAND          MCISENDCOMMAND
 0005:1386 MCISENDSTRING           MCISENDSTRING
 0005:2D6E MCISETDRIVERDATA        MCISETDRIVERDATA
 0005:2E30 MCISETYIELDPROC         MCISETYIELDPROC
 0006:0806 MIDIINADDBUFFER         MIDIINADDBUFFER
 0006:06C2 MIDIINCLOSE             MIDIINCLOSE
 0006:055C MIDIINGETDEVCAPS        MIDIINGETDEVCAPS
 0006:05A8 MIDIINGETERRORTEXT      MIDIINGETERRORTEXT
 0006:090C MIDIINGETID             MIDIINGETID
 0006:0506 MIDIINGETNUMDEVS        MIDIINGETNUMDEVS
 0006:0524 MIDIINMESSAGE           MIDIINMESSAGE
 0006:05E8 MIDIINOPEN              MIDIINOPEN
 0006:070A MIDIINPREPAREHEADER     MIDIINPREPAREHEADER
 0006:08D8 MIDIINRESET             MIDIINRESET
 0006:0870 MIDIINSTART             MIDIINSTART
 0006:08A4 MIDIINSTOP              MIDIINSTOP
 0006:0788 MIDIINUNPREPAREHEADER   MIDIINUNPREPAREHEADER
 0006:0494 MIDIOUTCACHEDRUMPATCHES  MIDIOUTCACHEDRUMPATCHES
 0006:0422 MIDIOUTCACHEPATCHES     MIDIOUTCACHEPATCHES
 0006:02DE MIDIOUTCLOSE            MIDIOUTCLOSE
 0006:00D2 MIDIOUTGETDEVCAPS       MIDIOUTGETDEVCAPS
 0006:01C4 MIDIOUTGETERRORTEXT     MIDIOUTGETERRORTEXT
 0006:0956 MIDIOUTGETID            MIDIOUTGETID
 0006:00B4 MIDIOUTGETNUMDEVS       MIDIOUTGETNUMDEVS
 0006:011E MIDIOUTGETVOLUME        MIDIOUTGETVOLUME
 0001:01B2 MIDIOUTLONGMSG          MIDIOUTLONGMSG
 0001:0146 MIDIOUTMESSAGE          MIDIOUTMESSAGE
 0006:0204 MIDIOUTOPEN             MIDIOUTOPEN
 0006:0326 MIDIOUTPREPAREHEADER    MIDIOUTPREPAREHEADER
 0001:0222 MIDIOUTRESET            MIDIOUTRESET
 0006:015E MIDIOUTSETVOLUME        MIDIOUTSETVOLUME
 0001:017C MIDIOUTSHORTMSG         MIDIOUTSHORTMSG
 0006:03A4 MIDIOUTUNPREPAREHEADER  MIDIOUTUNPREPAREHEADER
 0009:0738 MIXERCLOSE              MIXERCLOSE
 0009:0EF0 MIXERGETCONTROLDETAILS  MIXERGETCONTROLDETAILS
 0009:00E6 MIXERGETDEVCAPS         MIXERGETDEVCAPS
 0009:018A MIXERGETID              MIXERGETID
 0009:0D68 MIXERGETLINECONTROLS    MIXERGETLINECONTROLS
 0009:086E MIXERGETLINEINFO        MIXERGETLINEINFO
 0009:00C4 MIXERGETNUMDEVS         MIXERGETNUMDEVS
 0009:07D8 MIXERMESSAGE            MIXERMESSAGE
 0009:0562 MIXEROPEN               MIXEROPEN
 0009:10DC MIXERSETCONTROLDETAILS  MIXERSETCONTROLDETAILS
 0002:02D4 MMDRVINSTALL            MMDRVINSTALL
 0004:05D1 MMGETCURRENTTASK        MMGETCURRENTTASK
 0007:0D92 MMIOADVANCE             MMIOADVANCE
 0007:1590 MMIOASCEND              MMIOASCEND
 0007:0454 MMIOCLOSE               MMIOCLOSE
 0007:16D2 MMIOCREATECHUNK         MMIOCREATECHUNK
 0007:139C MMIODESCEND             MMIODESCEND
 0007:0CC2 MMIOFLUSH               MMIOFLUSH
 0007:092A MMIOGETINFO             MMIOGETINFO
 0007:0F52 MMIOINSTALLIOPROC       MMIOINSTALLIOPROC
 0007:02B8 MMIOOPEN                MMIOOPEN
 0007:04AE MMIOREAD                MMIOREAD
 0007:01E4 MMIORENAME              MMIORENAME
 0007:07E2 MMIOSEEK                MMIOSEEK
 0007:1098 MMIOSENDMESSAGE         MMIOSENDMESSAGE
 0007:0A62 MMIOSETBUFFER           MMIOSETBUFFER
 0007:0994 MMIOSETINFO             MMIOSETINFO
 0007:0EBA MMIOSTRINGTOFOURCC      MMIOSTRINGTOFOURCC
 0007:0624 MMIOWRITE               MMIOWRITE
 0002:02C8 MMSYSTEMGETVERSION      MMSYSTEMGETVERSION
 0004:05D6 MMTASKBLOCK             MMTASKBLOCK
 0004:0612 MMTASKCREATE            MMTASKCREATE
 0001:02D2 MMTASKSIGNAL            MMTASKSIGNAL
 0004:05B0 MMTASKYIELD             MMTASKYIELD
 0001:0374 OUTPUTDEBUGSTR          OUTPUTDEBUGSTR
 0004:0000 SNDPLAYSOUND            SNDPLAYSOUND
 0001:038C STACKENTER              STACKENTER
 0001:03E1 STACKLEAVE              STACKLEAVE
 0001:00AE TIMEBEGINPERIOD         TIMEBEGINPERIOD
 0001:00DA TIMEENDPERIOD           TIMEENDPERIOD
 0008:0000 TIMEGETDEVCAPS          TIMEGETDEVCAPS
 0001:0000 TIMEGETSYSTEMTIME       TIMEGETSYSTEMTIME
 0001:012E TIMEGETTIME             TIMEGETTIME
 0001:0106 TIMEKILLEVENT           TIMEKILLEVENT
 0001:0034 TIMESETEVENT            TIMESETEVENT
 0003:0D0C WAVEINADDBUFFER         WAVEINADDBUFFER
 0003:0BD2 WAVEINCLOSE             WAVEINCLOSE
 0003:0A0A WAVEINGETDEVCAPS        WAVEINGETDEVCAPS
 0003:0A56 WAVEINGETERRORTEXT      WAVEINGETERRORTEXT
 0003:0E5A WAVEINGETID             WAVEINGETID
 0003:09B6 WAVEINGETNUMDEVS        WAVEINGETNUMDEVS
 0003:0E0A WAVEINGETPOSITION       WAVEINGETPOSITION
 0003:09D4 WAVEINMESSAGE           WAVEINMESSAGE
 0003:0A96 WAVEINOPEN              WAVEINOPEN
 0003:0C14 WAVEINPREPAREHEADER     WAVEINPREPAREHEADER
 0003:0DD8 WAVEINRESET             WAVEINRESET
 0003:0D74 WAVEINSTART             WAVEINSTART
 0003:0DA6 WAVEINSTOP              WAVEINSTOP
 0003:0C90 WAVEINUNPREPAREHEADER   WAVEINUNPREPAREHEADER
 0003:0830 WAVEOUTBREAKLOOP        WAVEOUTBREAKLOOP
 0003:05EC WAVEOUTCLOSE            WAVEOUTCLOSE
 0003:037E WAVEOUTGETDEVCAPS       WAVEOUTGETDEVCAPS
 0003:0470 WAVEOUTGETERRORTEXT     WAVEOUTGETERRORTEXT
 0003:0EA4 WAVEOUTGETID            WAVEOUTGETID
 0003:032A WAVEOUTGETNUMDEVS       WAVEOUTGETNUMDEVS
 0003:08B2 WAVEOUTGETPITCH         WAVEOUTGETPITCH
 0003:0934 WAVEOUTGETPLAYBACKRATE  WAVEOUTGETPLAYBACKRATE
 0003:0862 WAVEOUTGETPOSITION      WAVEOUTGETPOSITION
 0003:03CA WAVEOUTGETVOLUME        WAVEOUTGETVOLUME
 0003:0348 WAVEOUTMESSAGE          WAVEOUTMESSAGE
 0003:04B0 WAVEOUTOPEN             WAVEOUTOPEN
 0003:079A WAVEOUTPAUSE            WAVEOUTPAUSE
 0003:062E WAVEOUTPREPAREHEADER    WAVEOUTPREPAREHEADER
 0003:07FE WAVEOUTRESET            WAVEOUTRESET
 0003:07CC WAVEOUTRESTART          WAVEOUTRESTART
 0003:0900 WAVEOUTSETPITCH         WAVEOUTSETPITCH
 0003:0982 WAVEOUTSETPLAYBACKRATE  WAVEOUTSETPLAYBACKRATE
 0003:040A WAVEOUTSETVOLUME        WAVEOUTSETVOLUME
 0003:06B2 WAVEOUTUNPREPAREHEADER  WAVEOUTUNPREPAREHEADER
 0003:072E WAVEOUTWRITE            WAVEOUTWRITE
 0002:0014 WEP                     WEP

  Address         Publics by Name

 0000:0000  Imp  ANSILOWER            (USER.432)
 0000:0000  Imp  ANSIUPPER            (USER.431)
 0004:00DC       APPEXIT
 000B:0238       AUX32MESSAGE
 0008:058C       AUXGETDEVCAPS
 0008:0572       AUXGETNUMDEVS
 0008:05D4       AUXGETVOLUME
 0008:0632       AUXOUTMESSAGE
 0008:0610       AUXSETVOLUME
 0004:06A2       BWINEXEC
 0000:0000  Imp  CALLPROC32W          (KERNEL.517)
 000B:00F0       CB32
 0001:0560       CheckThunkInit
 0000:0000  Imp  CLOSEDRIVER          (USER.253)
 0001:038A       CodeFixDS
 0001:0388       CodeFixWinFlags
 0005:1626       COULDBE16BITDRV
 0000:0000  Imp  CREATEWINDOWEX       (USER.452)
 0000:0000  Imp  DEFDRIVERPROC        (USER.255)
 0000:0000  Imp  DEFWINDOWPROC        (USER.107)
 0001:070A       DEINSTALLINTERRUPTHANDLER
 0000:0000  Imp  DispatchMessage      (USER.114)
 0001:0413       DoInterrupt
 0005:3E86       DOSCHANGEDIR
 0005:3F2A       DOSGETCURRENTDIR
 0005:3F06       DOSGETCURRENTDRIVE
 0005:3F0D       DOSSETCURRENTDRIVE
 0001:049E       DRIVERCALLBACK
 0004:0036       DRIVERPROC
 0004:059B       DRVCLOSE
 0004:05AA       DRVDEFDRIVERPROC
 0002:0188       DRVFREE
 0004:05A0       DRVGETMODULEHANDLE
 0002:01A2       DRVLOAD
 0004:0596       DRVOPEN
 0004:05A5       DRVSENDMESSAGE
 0005:342A       FINDCOMMANDINTABLE
 0005:3518       FINDCOMMANDITEM
 0000:0000  Imp  FINDRESOURCE         (KERNEL.60)
 0004:0333       FREEHANDLE
 0000:0000  Imp  FREELIBRARY          (KERNEL.96)
 0000:0000  Imp  FREERESOURCE         (KERNEL.63)
 0007:17AA       FSTRRCHR
 0000:0000  Imp  GETACTIVEWINDOW      (USER.60)
 0000:0000  Imp  GETASYNCKEYSTATE     (USER.249)
 0000:0000  Imp  GetCodeInfo          (KERNEL.104)
 0000:0000  Imp  GETCURRENTTASK       (KERNEL.36)
 0000:0000  Imp  GETDRIVERMODULEHANDLE (USER.254)
 0000:0000  Imp  GetLPErrMode         (KERNEL.99)
 0000:0000  Imp  GetMessage           (USER.108)
 0000:0000  Imp  GETPRIVATEPROFILEINT (KERNEL.127)
 0000:0000  Imp  GETPRIVATEPROFILESTRING (KERNEL.128)
 0000:0000  Imp  GETPROCADDRESS       (KERNEL.50)
 0000:0000  Imp  GETPROCADDRESS32W    (KERNEL.515)
 0000:0000  Imp  GETPROFILESTRING     (KERNEL.58)
 0000:0000  Imp  GETTEMPFILENAME      (KERNEL.97)
 0000:0000  Imp  GETWINDOWTASK        (USER.224)
 0000:0000  Imp  GLOBALALLOC          (KERNEL.15)
 0000:0000  Imp  GlobalFix            (KERNEL.197)
 0000:0000  Imp  GLOBALFREE           (KERNEL.17)
 0000:0000  Imp  GlobalHandle         (KERNEL.21)
 0000:0000  Imp  GlobalHandleNoRip    (KERNEL.159)
 0000:0000  Imp  GLOBALLOCK           (KERNEL.18)
 0000:0000  Imp  GLOBALPAGELOCK       (KERNEL.191)
 0000:0000  Imp  GLOBALPAGEUNLOCK     (KERNEL.192)
 0000:0000  Imp  GLOBALREALLOC        (KERNEL.16)
 0000:0000  Imp  GlobalUnFix          (KERNEL.198)
 0000:0000  Imp  GLOBALUNLOCK         (KERNEL.19)
 000A:0002       GWSTACKFRAMES
 000A:0006       GWSTACKSELECTOR
 000A:0000       GWSTACKSIZE
 000A:0004       GWSTACKUSE
 0005:00AA       HANDLENOTIFY
 000A:0008       HDRVDESTROY
 0005:3E2E       HEAPALLOC
 0002:07AA       HEAPCREATE
 0002:07E5       HEAPDESTROY
 0005:3E6F       HEAPFREE
 0005:3E4E       HEAPREALLOC
 000A:000E       HGLOBAL
 0004:0798       HUGEPAGELOCK
 0004:07C4       HUGEPAGEUNLOCK
 0009:01C6       IMIXERGETID
 0009:0000       IMIXERMAPID
 0009:0040       IMIXERMESSAGEHANDLE
 0009:006A       IMIXERMESSAGEID
 0009:12DC       INITMIXERTHUNKS
 0001:05D6       INSTALLINTERRUPTHANDLER
 0005:1692       IS16BITDRV
 0000:0000  Imp  IsBadCodePtr         (KERNEL.336)
 0000:0000  Imp  IsBadHugeReadPtr     (KERNEL.346)
 0000:0000  Imp  IsBadHugeWritePtr    (KERNEL.347)
 0000:0000  Imp  IsBadReadPtr         (KERNEL.334)
 0000:0000  Imp  IsBadStringPtr       (KERNEL.337)
 0000:0000  Imp  IsBadWritePtr        (KERNEL.335)
 0000:0000  Imp  IsSharedSelector     (KERNEL.345)
 0000:0000  Imp  IsTask               (KERNEL.320)
 0000:0000  Imp  ISTASKLOCKED         (KERNEL.122)
 0000:0000  Imp  ISWINDOW             (USER.47)
 000B:0228       JOY32MESSAGE
 0008:0022       JOYGETDEVCAPS
 0008:008C       JOYGETNUMDEVS
 0008:00A8       JOYGETPOS
 0008:0112       JOYGETTHRESHOLD
 0002:0666       JOYINIT
 0008:0670       JOYMESSAGE
 0008:03DE       JOYPOLLCALLBACK
 0008:0176       JOYRELEASECAPTURE
 0008:0318       JOYSETCALIBRATION
 0008:01DE       JOYSETCAPTURE
 0008:02CE       JOYSETTHRESHOLD
 0000:0000  Imp  KILLTIMER            (USER.12)
 0002:0000       LibEntry
 0002:001A       LibMain
 0000:0000  Imp  LOADLIBRARY          (KERNEL.95)
 0000:0000  Imp  LOADLIBRARYEX32W     (KERNEL.513)
 0000:0000  Imp  LoadModule           (KERNEL.45)
 0000:0000  Imp  LOADRESOURCE         (KERNEL.61)
 0000:0000  Imp  LOADSTRING           (USER.176)
 0000:0000  Imp  LOCALALLOC           (KERNEL.5)
 0000:0000  Imp  LocalCompact         (KERNEL.13)
 0000:0000  Imp  LocalCountFree       (KERNEL.161)
 0000:0000  Imp  LOCALFREE            (KERNEL.7)
 0000:0000  Imp  LocalHeapSize        (KERNEL.162)
 0000:0000  Imp  LocalInit            (KERNEL.4)
 0000:0000  Imp  LocalReAlloc         (KERNEL.6)
 0000:0000  Imp  LOCALSHRINK          (KERNEL.121)
 0000:0000  Imp  LOCKRESOURCE         (KERNEL.62)
 0000:0000  Imp  LOGPARAMERROR        (KERNEL.325)
 0000:0000  Imp  LSTRCMP              (USER.430)
 0000:0000  Imp  LSTRCMPI             (USER.471)
 0000:0000  Imp  LSTRCPY              (KERNEL.88)
 0000:0000  Imp  LSTRCPYN             (KERNEL.353)
 0000:0000  Imp  LSTRLEN              (KERNEL.90)
 000B:021C       MCI32MESSAGE
 0005:1DAA       MCIADDDEVICENAME
 0005:1DFA       MCIALLOCATENODE
 0005:0142       MCIAUTOCLOSEDEVICE
 0005:0C42       MCIAUTOOPENDEVICE
 0005:00E0       MCIBREAK
 0005:2F34       MCIBREAKKEYYIELDPROC
 0005:35FA       MCICHECKTOKEN
 0005:2C76       MCICLOSEDEVICE
 0005:06F2       MCICOLONIZE
 0005:0660       MCICOLONIZEDIGIT
 0005:0778       MCICONVERTRETURNVALUE
 0005:194C       MCIDEVICEMATCH
 0001:02E3       MCIDRIVERNOTIFY
 0005:2DC6       MCIDRIVERYIELD
 0005:2FA6       MCIEATCOMMANDENTRY
 0005:2630       MCIEATTOKEN
 0005:146C       MCIEXECUTE
 0005:259E       MCIEXTRACTDEVICETYPE
 0005:27C6       MCIEXTRACTTYPEFROMID
 0005:2032       MCIFINDDRIVERNAME
 0005:0BBA       MCIFINDNOTIFY
 0005:3348       MCIFREECOMMANDRESOURCE
 0005:1906       MCIGETCREATORTASK
 0005:188A       MCIGETDEVICEID
 0005:1718       MCIGETDEVICEIDFROMELEMENTID
 0005:17E6       MCIGETDEVICEIDINTERNAL
 0005:18CE       MCIGETDEVICEIDINTERNALEX
 0005:2D1E       MCIGETDRIVERDATA
 0005:155A       MCIGETERRORSTRING
 0005:3022       MCIGETPARAMSIZE
 0005:2EAA       MCIGETYIELDPROC
 0005:16E2       MCIINITDEVICELIST
 0005:30CA       MCILOADCOMMANDRESOURCE
 0005:21E0       MCILOADDEVICE
 0005:32D4       MCILOADTABLETYPE
 0005:19D6       MCILOOKUPTYPE
 0005:3DF0       MCIMESSAGE
 0005:0050       MCINOTIFY
 0005:284E       MCIOPENDEVICE
 0005:3886       MCIPARSEARGUMENT
 0005:3D52       MCIPARSECOMMAND
 0005:37F0       MCIPARSECONSTANT
 0005:3690       MCIPARSEINTEGER
 0005:39F4       MCIPARSEPARAMS
 0005:3DA0       MCIPARSERFREE
 0005:306A       MCIREGISTERCOMMANDTABLE
 0005:0AF4       MCIRELAYSYSTEMSTRING
 0005:1E9C       MCIREPARSEOPEN
 0005:04E6       MCISENDCOMMAND
 0005:05EE       MCISENDCOMMAND16
 0005:030E       MCISENDCOMMANDINTERNAL
 0005:01B0       MCISENDSINGLECOMMAND
 0005:1386       MCISENDSTRING
 0005:0DB0       MCISENDSTRINGINTERNAL
 0005:09FC       MCISENDSYSTEMSTRING
 0005:0912       MCISEPARATECOMMANDPARTS
 0005:2F8C       MCISETBREAKKEY
 0005:2D6E       MCISETDRIVERDATA
 0005:2E30       MCISETYIELDPROC
 0005:1A1C       MCISYSINFO
 0002:06C4       MCITERMINATE
 0005:3412       MCIUNLOCKCOMMANDTABLE
 0007:17DB       MEMCOPY
 0007:182C       MemCopy286
 0007:17E6       MemCopy386
 0000:0000  Imp  MESSAGEBOX           (USER.1)
 000B:0224       MID32MESSAGE
 0006:09D7       MIDIIIDMESSAGE
 0001:0335       MIDIIMESSAGE
 0006:0806       MIDIINADDBUFFER
 0006:06C2       MIDIINCLOSE
 0006:055C       MIDIINGETDEVCAPS
 0006:05A8       MIDIINGETERRORTEXT
 0006:090C       MIDIINGETID
 0006:0506       MIDIINGETNUMDEVS
 0006:0524       MIDIINMESSAGE
 0006:05E8       MIDIINOPEN
 0006:070A       MIDIINPREPAREHEADER
 0006:08D8       MIDIINRESET
 0006:0870       MIDIINSTART
 0006:08A4       MIDIINSTOP
 0006:0788       MIDIINUNPREPAREHEADER
 0006:0000       MIDILOCKDATA
 0006:09A0       MIDIOIDMESSAGE
 0001:02F6       MIDIOMESSAGE
 0006:0494       MIDIOUTCACHEDRUMPATCHES
 0006:0422       MIDIOUTCACHEPATCHES
 0006:02DE       MIDIOUTCLOSE
 0006:00D2       MIDIOUTGETDEVCAPS
 0006:01C4       MIDIOUTGETERRORTEXT
 0006:0956       MIDIOUTGETID
 0006:00B4       MIDIOUTGETNUMDEVS
 0006:011E       MIDIOUTGETVOLUME
 0001:01B2       MIDIOUTLONGMSG
 0001:0146       MIDIOUTMESSAGE
 0006:0204       MIDIOUTOPEN
 0006:0326       MIDIOUTPREPAREHEADER
 0001:0222       MIDIOUTRESET
 0006:015E       MIDIOUTSETVOLUME
 0001:017C       MIDIOUTSHORTMSG
 0006:03A4       MIDIOUTUNPREPAREHEADER
 0006:0024       MIDIUNLOCKDATA
 0009:0738       MIXERCLOSE
 0009:0EF0       MIXERGETCONTROLDETAILS
 0009:00E6       MIXERGETDEVCAPS
 0009:018A       MIXERGETID
 0009:0D68       MIXERGETLINECONTROLS
 0009:086E       MIXERGETLINEINFO
 0009:00C4       MIXERGETNUMDEVS
 0009:07D8       MIXERMESSAGE
 0009:0562       MIXEROPEN
 0009:10DC       MIXERSETCONTROLDETAILS
 0001:05C9       MMCALLPROC32
 0002:02D4       MMDRVINSTALL
 0002:0378       MMDRVOPEN
 0004:05D1       MMGETCURRENTTASK
 0007:0D92       MMIOADVANCE
 0007:1590       MMIOASCEND
 0007:0454       MMIOCLOSE
 0007:16D2       MMIOCREATECHUNK
 0007:139C       MMIODESCEND
 0007:0CC2       MMIOFLUSH
 0007:092A       MMIOGETINFO
 0007:0F52       MMIOINSTALLIOPROC
 0007:02B8       MMIOOPEN
 0007:04AE       MMIOREAD
 0007:01E4       MMIORENAME
 0007:07E2       MMIOSEEK
 0007:1098       MMIOSENDMESSAGE
 0007:0A62       MMIOSETBUFFER
 0007:0994       MMIOSETINFO
 0007:0EBA       MMIOSTRINGTOFOURCC
 0007:0624       MMIOWRITE
 0002:02C8       MMSYSTEMGETVERSION
 0004:05D6       MMTASKBLOCK
 0004:0612       MMTASKCREATE
 0001:02D2       MMTASKSIGNAL
 0004:05B0       MMTASKYIELD
 000A:0016       MMWOW32LIB
 000B:0220       MOD32MESSAGE
 0009:13A6       MXDMESSAGE
 0004:02FE       NEWHANDLE
 0008:06A9       NOTIFY_CALLBACK_DATA
 0000:0000  Imp  OEMTOANSI            (KEYBOARD.6)
 0000:0000  Imp  OPENDRIVER           (USER.252)
 0000:0000  Imp  OPENFILE             (KERNEL.74)
 0001:0374       OUTPUTDEBUGSTR
 0000:0000  Imp  OutputDebugString    (KERNEL.115)
 000B:0008       pAtomTable
 0000:0000  Imp  PEEKMESSAGE          (USER.109)
 000B:0006       pLocalHeap
 0000:0000  Imp  PostAppMessage       (USER.116)
 0000:0000  Imp  POSTMESSAGE          (USER.110)
 000B:000E       pStackBot
 000B:000C       pStackMin
 000B:000A       pStackTop
 0000:0000  Imp  REGISTERCLASS        (USER.57)
 000B:0006       rsrvptrs
 0000:0000  Imp  SENDDRIVERMESSAGE    (USER.251)
 0000:0000  Imp  SENDMESSAGE          (USER.111)
 0000:0000  Imp  SETTIMER             (USER.10)
 0003:0232       SNDMESSAGE
 0004:0000       SNDPLAYSOUND
 0003:009A       SNDPLAYSOUNDI
 0003:1016       SOUNDCLOSE
 0003:108C       SOUNDFREE
 0003:1202       SOUNDINITWAVHDR
 0003:10A6       SOUNDLOADFILE
 0003:11A4       SOUNDLOADMEMORY
 0003:0F30       SOUNDOPEN
 0003:0F06       SOUNDPLAY
 0003:1074       SOUNDWAIT
 0001:038C       STACKENTER
 0002:01BC       STACKINIT
 0001:03E1       STACKLEAVE
 0002:029A       STACKTERMINATE
 0002:03BA       THUNKINIT
 000A:0012       TID32MESSAGE
 0001:00AE       TIMEBEGINPERIOD
 0001:00DA       TIMEENDPERIOD
 0008:0000       TIMEGETDEVCAPS
 0001:0000       TIMEGETSYSTEMTIME
 0001:012E       TIMEGETTIME
 0002:0548       TIMEINIT
 0001:0106       TIMEKILLEVENT
 0001:057B       TIMEMESSAGE
 0001:0034       TIMESETEVENT
 0000:0000  Imp  TranslateMessage     (USER.113)
 0000:0000  Imp  UNREGISTERCLASS      (USER.403)
 0004:0534       VALIDATECALLBACK
 0004:0506       VALIDATEDRIVERCALLBACK
 0001:0256       VALIDATEHANDLE
 0004:036B       VALIDATEHEADER
 0004:0425       VALIDATEREADPOINTER
 0004:0563       VALIDATESTRING
 0001:028C       VALIDATETIMERCALLBACK
 0004:045A       VALIDATEWRITEPOINTER
 000A:000A       VPCALLBACKDATA
 0005:1D32       WADDDEVICENODETOLIST
 0003:14A1       WAVEIIDMESSAGE
 0003:1439       WAVEIMESSAGE
 0003:0D0C       WAVEINADDBUFFER
 0003:0BD2       WAVEINCLOSE
 0003:0A0A       WAVEINGETDEVCAPS
 0003:0A56       WAVEINGETERRORTEXT
 0003:0E5A       WAVEINGETID
 0003:09B6       WAVEINGETNUMDEVS
 0003:0E0A       WAVEINGETPOSITION
 0003:09D4       WAVEINMESSAGE
 0003:0A96       WAVEINOPEN
 0003:0C14       WAVEINPREPAREHEADER
 0003:0DD8       WAVEINRESET
 0003:0D74       WAVEINSTART
 0003:0DA6       WAVEINSTOP
 0003:0C90       WAVEINUNPREPAREHEADER
 0003:13D4       WAVEOIDMESSAGE
 0003:136C       WAVEOMESSAGE
 0003:0830       WAVEOUTBREAKLOOP
 0003:05EC       WAVEOUTCLOSE
 0003:037E       WAVEOUTGETDEVCAPS
 0003:0470       WAVEOUTGETERRORTEXT
 0003:0EA4       WAVEOUTGETID
 0003:032A       WAVEOUTGETNUMDEVS
 0003:08B2       WAVEOUTGETPITCH
 0003:0934       WAVEOUTGETPLAYBACKRATE
 0003:0862       WAVEOUTGETPOSITION
 0003:03CA       WAVEOUTGETVOLUME
 0003:0348       WAVEOUTMESSAGE
 0003:0EEE       WAVEOUTNOTIFY
 0003:04B0       WAVEOUTOPEN
 0003:079A       WAVEOUTPAUSE
 0003:062E       WAVEOUTPREPAREHEADER
 0003:07FE       WAVEOUTRESET
 0003:07CC       WAVEOUTRESTART
 0003:0900       WAVEOUTSETPITCH
 0003:0982       WAVEOUTSETPLAYBACKRATE
 0003:040A       WAVEOUTSETVOLUME
 0003:06B2       WAVEOUTUNPREPAREHEADER
 0003:072E       WAVEOUTWRITE
 0002:0014       WEP
 000B:0230       WID32MESSAGE
 000B:00F8       WIDMAPPER
 0002:0730       WNDINIT
 0002:0784       WNDTERMINATE
 000B:022C       WOD32MESSAGE
 000B:00F4       WODMAPPER
 0000:0000  Imp  WOW16Call            (KERNEL.500)
 0000:0000  Imp  wvsprintf            (USER.421)
 0000:0000  Imp  YIELD                (KERNEL.29)
 000B:0104       _command_tables
 0000:0000  Imp  _DebugOutput         (KERNEL.328)
 000B:0100       _ghInst
 000B:0062       _gIOProcMapHead
 000B:0072       _gpMixerDevHeader
 000B:00E8       _guTotalMixerDevs
 000B:00FC       _hMciHeap
 0000:0000  Imp  _HREAD               (KERNEL.349)
 000B:00FE       _hwndNotify
 0000:0000  Imp  _HWRITE              (KERNEL.350)
 0000:0000  Imp  _LCLOSE              (KERNEL.81)
 0000:0000  Imp  _LLSEEK              (KERNEL.84)
 000B:0242       _lpWavHdr
 0005:0000       _mciAppExit
 000B:00EA       _MCI_bDeviceListInitialized
 000B:00EC       _MCI_lpDeviceList
 000B:023C       _MCI_wDeviceListSize
 000B:0042       _MCI_wNextDeviceID
 000B:0234       _mix32Lib
 000B:023E       _mix32Message
 000B:00E0       _mixerdrv
 000B:0102       _pHandleList
 0002:016F       _szBoot
 0002:0164       _szDriverProc
 0002:0174       _szDrivers
 000B:001E       _szJoyKey
 0002:015B       _szJoystick
 0002:014E       _szJoystickDrv
 0002:013F       _szMMSystem
 0002:0187       _szNull
 0005:004B       _szOpen
 0002:0133       _szStackFrames
 0002:0129       _szStackSize
 0002:0724       _szStartupSound
 0003:0083       _szSystemDefault
 0002:017C       _szSystemIni
 0002:0148       _szTimerDrv
 0000:0000  Imp  _wsprintf            (USER.420)
 0000:0001  Abs  __acrtused
 0004:0812       __aFahdiff
 0004:0832       __aFFalmul
 0004:0832       __aFFaulmul
 0004:0854       __aFlmul
 0004:0854       __aFulmul
 0000:0000  Imp  __AHINCR             (KERNEL.114)
 0000:0000  Imp  __AHSHIFT            (KERNEL.113)
 0004:0886       __fstrstr
 0000:0000  Imp  __MOD_COMMDLG        (KERNEL.532)
 0000:0000  Imp  __MOD_DGDI           (KERNEL.525)
 0000:0000  Imp  __MOD_DKERNEL        (KERNEL.521)
 0000:0000  Imp  __MOD_DUSER          (KERNEL.523)
 0000:0000  Imp  __MOD_GDI            (KERNEL.524)
 0000:0000  Imp  __MOD_KERNEL         (KERNEL.520)
 0000:0000  Imp  __MOD_KEYBOARD       (KERNEL.526)
 0000:0000  Imp  __MOD_MMEDIA         (KERNEL.531)
 0000:0000  Imp  __MOD_SHELL          (KERNEL.528)
 0000:0000  Imp  __MOD_SOUND          (KERNEL.527)
 0000:0000  Imp  __MOD_TOOLHELP       (KERNEL.530)
 0000:0000  Imp  __MOD_USER           (KERNEL.522)
 0000:0000  Imp  __MOD_WINSOCK        (KERNEL.529)
 0000:0000  Imp  __WINFLAGS           (KERNEL.178)

  Address         Publics by Value

 0000:0000  Imp  KILLTIMER            (USER.12)
 0000:0000  Imp  _HREAD               (KERNEL.349)
 0000:0000  Imp  LOADLIBRARYEX32W     (KERNEL.513)
 0000:0000  Imp  GLOBALUNLOCK         (KERNEL.19)
 0000:0000  Imp  GETCURRENTTASK       (KERNEL.36)
 0000:0000  Imp  OPENDRIVER           (USER.252)
 0000:0000  Imp  LSTRLEN              (KERNEL.90)
 0000:0000  Imp  GetLPErrMode         (KERNEL.99)
 0000:0000  Imp  GETDRIVERMODULEHANDLE (USER.254)
 0000:0000  Imp  _DebugOutput         (KERNEL.328)
 0000:0000  Imp  _LCLOSE              (KERNEL.81)
 0000:0000  Imp  GETPRIVATEPROFILEINT (KERNEL.127)
 0000:0000  Imp  LocalHeapSize        (KERNEL.162)
 0000:0000  Imp  TranslateMessage     (USER.113)
 0000:0000  Imp  __MOD_DGDI           (KERNEL.525)
 0000:0000  Imp  GLOBALFREE           (KERNEL.17)
 0000:0000  Imp  GlobalUnFix          (KERNEL.198)
 0000:0000  Imp  __AHINCR             (KERNEL.114)
 0000:0000  Imp  UNREGISTERCLASS      (USER.403)
 0000:0000  Imp  LSTRCMP              (USER.430)
 0000:0000  Imp  __MOD_SHELL          (KERNEL.528)
 0000:0000  Imp  LOCALFREE            (KERNEL.7)
 0000:0000  Imp  GETACTIVEWINDOW      (USER.60)
 0000:0000  Imp  WOW16Call            (KERNEL.500)
 0000:0000  Imp  __MOD_DUSER          (KERNEL.523)
 0000:0000  Imp  _HWRITE              (KERNEL.350)
 0000:0000  Imp  GLOBALPAGEUNLOCK     (KERNEL.192)
 0000:0000  Imp  OPENFILE             (KERNEL.74)
 0000:0000  Imp  DispatchMessage      (USER.114)
 0000:0000  Imp  __AHSHIFT            (KERNEL.113)
 0000:0000  Imp  LSTRCPY              (KERNEL.88)
 0000:0000  Imp  GLOBALALLOC          (KERNEL.15)
 0000:0000  Imp  CREATEWINDOWEX       (USER.452)
 0000:0000  Imp  MESSAGEBOX           (USER.1)
 0000:0000  Imp  IsBadHugeWritePtr    (KERNEL.347)
 0000:0000  Imp  ANSILOWER            (USER.432)
 0000:0000  Imp  __MOD_KEYBOARD       (KERNEL.526)
 0000:0000  Imp  GLOBALREALLOC        (KERNEL.16)
 0000:0000  Imp  FINDRESOURCE         (KERNEL.60)
 0000:0000  Imp  LocalReAlloc         (KERNEL.6)
 0000:0000  Imp  __WINFLAGS           (KERNEL.178)
 0000:0000  Imp  wvsprintf            (USER.421)
 0000:0000  Imp  IsSharedSelector     (KERNEL.345)
 0000:0000  Imp  GETPRIVATEPROFILESTRING (KERNEL.128)
 0000:0000  Imp  LOCALSHRINK          (KERNEL.121)
 0000:0000  Imp  LOGPARAMERROR        (KERNEL.325)
 0000:0000  Imp  GetMessage           (USER.108)
 0000:0000  Imp  __MOD_KERNEL         (KERNEL.520)
 0000:0000  Imp  GETPROCADDRESS32W    (KERNEL.515)
 0000:0000  Imp  LocalInit            (KERNEL.4)
 0000:0000  Imp  CLOSEDRIVER          (USER.253)
 0000:0000  Imp  LoadModule           (KERNEL.45)
 0000:0000  Imp  LocalCountFree       (KERNEL.161)
 0000:0000  Imp  POSTMESSAGE          (USER.110)
 0000:0000  Imp  GlobalHandleNoRip    (KERNEL.159)
 0000:0000  Imp  LSTRCMPI             (USER.471)
 0000:0000  Imp  SETTIMER             (USER.10)
 0000:0000  Imp  DEFWINDOWPROC        (USER.107)
 0000:0000  Imp  IsBadStringPtr       (KERNEL.337)
 0000:0000  Imp  __MOD_GDI            (KERNEL.524)
 0000:0000  Imp  LSTRCPYN             (KERNEL.353)
 0000:0000  Imp  __MOD_WINSOCK        (KERNEL.529)
 0000:0000  Imp  SENDMESSAGE          (USER.111)
 0000:0000  Imp  GlobalFix            (KERNEL.197)
 0000:0000  Imp  OEMTOANSI            (KEYBOARD.6)
 0000:0000  Imp  GETTEMPFILENAME      (KERNEL.97)
 0000:0000  Imp  FREERESOURCE         (KERNEL.63)
 0000:0000  Imp  ISWINDOW             (USER.47)
 0000:0000  Imp  PostAppMessage       (USER.116)
 0000:0000  Imp  GETASYNCKEYSTATE     (USER.249)
 0000:0000  Imp  GlobalHandle         (KERNEL.21)
 0000:0000  Imp  SENDDRIVERMESSAGE    (USER.251)
 0000:0000  Imp  GETPROFILESTRING     (KERNEL.58)
 0000:0000  Imp  PEEKMESSAGE          (USER.109)
 0000:0000  Imp  __MOD_USER           (KERNEL.522)
 0000:0000  Imp  LOADSTRING           (USER.176)
 0000:0000  Imp  IsTask               (KERNEL.320)
 0000:0000  Imp  GetCodeInfo          (KERNEL.104)
 0000:0000  Imp  LOCALALLOC           (KERNEL.5)
 0000:0000  Imp  REGISTERCLASS        (USER.57)
 0000:0000  Imp  YIELD                (KERNEL.29)
 0000:0000  Imp  __MOD_COMMDLG        (KERNEL.532)
 0000:0000  Imp  LocalCompact         (KERNEL.13)
 0000:0000  Imp  DEFDRIVERPROC        (USER.255)
 0000:0000  Imp  GETPROCADDRESS       (KERNEL.50)
 0000:0000  Imp  ISTASKLOCKED         (KERNEL.122)
 0000:0000  Imp  GLOBALPAGELOCK       (KERNEL.191)
 0000:0000  Imp  GLOBALLOCK           (KERNEL.18)
 0000:0000  Imp  LOADRESOURCE         (KERNEL.61)
 0000:0000  Imp  IsBadWritePtr        (KERNEL.335)
 0000:0000  Imp  _LLSEEK              (KERNEL.84)
 0000:0000  Imp  LOADLIBRARY          (KERNEL.95)
 0000:0000  Imp  IsBadCodePtr         (KERNEL.336)
 0000:0000  Imp  __MOD_MMEDIA         (KERNEL.531)
 0000:0000  Imp  LOCKRESOURCE         (KERNEL.62)
 0000:0000  Imp  IsBadHugeReadPtr     (KERNEL.346)
 0000:0000  Imp  CALLPROC32W          (KERNEL.517)
 0000:0000  Imp  GETWINDOWTASK        (USER.224)
 0000:0000  Imp  IsBadReadPtr         (KERNEL.334)
 0000:0000  Imp  __MOD_SOUND          (KERNEL.527)
 0000:0000  Imp  _wsprintf            (USER.420)
 0000:0000  Imp  ANSIUPPER            (USER.431)
 0000:0000  Imp  __MOD_DKERNEL        (KERNEL.521)
 0000:0000  Imp  OutputDebugString    (KERNEL.115)
 0000:0000  Imp  FREELIBRARY          (KERNEL.96)
 0000:0000  Imp  __MOD_TOOLHELP       (KERNEL.530)
 0000:0001  Abs  __acrtused
 0001:0000       TIMEGETSYSTEMTIME
 0001:0034       TIMESETEVENT
 0001:00AE       TIMEBEGINPERIOD
 0001:00DA       TIMEENDPERIOD
 0001:0106       TIMEKILLEVENT
 0001:012E       TIMEGETTIME
 0001:0146       MIDIOUTMESSAGE
 0001:017C       MIDIOUTSHORTMSG
 0001:01B2       MIDIOUTLONGMSG
 0001:0222       MIDIOUTRESET
 0001:0256       VALIDATEHANDLE
 0001:028C       VALIDATETIMERCALLBACK
 0001:02D2       MMTASKSIGNAL
 0001:02E3       MCIDRIVERNOTIFY
 0001:02F6       MIDIOMESSAGE
 0001:0335       MIDIIMESSAGE
 0001:0374       OUTPUTDEBUGSTR
 0001:0388       CodeFixWinFlags
 0001:038A       CodeFixDS
 0001:038C       STACKENTER
 0001:03E1       STACKLEAVE
 0001:0413       DoInterrupt
 0001:049E       DRIVERCALLBACK
 0001:0560       CheckThunkInit
 0001:057B       TIMEMESSAGE
 0001:05C9       MMCALLPROC32
 0001:05D6       INSTALLINTERRUPTHANDLER
 0001:070A       DEINSTALLINTERRUPTHANDLER
 0002:0000       LibEntry
 0002:0014       WEP
 0002:001A       LibMain
 0002:0129       _szStackSize
 0002:0133       _szStackFrames
 0002:013F       _szMMSystem
 0002:0148       _szTimerDrv
 0002:014E       _szJoystickDrv
 0002:015B       _szJoystick
 0002:0164       _szDriverProc
 0002:016F       _szBoot
 0002:0174       _szDrivers
 0002:017C       _szSystemIni
 0002:0187       _szNull
 0002:0188       DRVFREE
 0002:01A2       DRVLOAD
 0002:01BC       STACKINIT
 0002:029A       STACKTERMINATE
 0002:02C8       MMSYSTEMGETVERSION
 0002:02D4       MMDRVINSTALL
 0002:0378       MMDRVOPEN
 0002:03BA       THUNKINIT
 0002:0548       TIMEINIT
 0002:0666       JOYINIT
 0002:06C4       MCITERMINATE
 0002:0724       _szStartupSound
 0002:0730       WNDINIT
 0002:0784       WNDTERMINATE
 0002:07AA       HEAPCREATE
 0002:07E5       HEAPDESTROY
 0003:0083       _szSystemDefault
 0003:009A       SNDPLAYSOUNDI
 0003:0232       SNDMESSAGE
 0003:032A       WAVEOUTGETNUMDEVS
 0003:0348       WAVEOUTMESSAGE
 0003:037E       WAVEOUTGETDEVCAPS
 0003:03CA       WAVEOUTGETVOLUME
 0003:040A       WAVEOUTSETVOLUME
 0003:0470       WAVEOUTGETERRORTEXT
 0003:04B0       WAVEOUTOPEN
 0003:05EC       WAVEOUTCLOSE
 0003:062E       WAVEOUTPREPAREHEADER
 0003:06B2       WAVEOUTUNPREPAREHEADER
 0003:072E       WAVEOUTWRITE
 0003:079A       WAVEOUTPAUSE
 0003:07CC       WAVEOUTRESTART
 0003:07FE       WAVEOUTRESET
 0003:0830       WAVEOUTBREAKLOOP
 0003:0862       WAVEOUTGETPOSITION
 0003:08B2       WAVEOUTGETPITCH
 0003:0900       WAVEOUTSETPITCH
 0003:0934       WAVEOUTGETPLAYBACKRATE
 0003:0982       WAVEOUTSETPLAYBACKRATE
 0003:09B6       WAVEINGETNUMDEVS
 0003:09D4       WAVEINMESSAGE
 0003:0A0A       WAVEINGETDEVCAPS
 0003:0A56       WAVEINGETERRORTEXT
 0003:0A96       WAVEINOPEN
 0003:0BD2       WAVEINCLOSE
 0003:0C14       WAVEINPREPAREHEADER
 0003:0C90       WAVEINUNPREPAREHEADER
 0003:0D0C       WAVEINADDBUFFER
 0003:0D74       WAVEINSTART
 0003:0DA6       WAVEINSTOP
 0003:0DD8       WAVEINRESET
 0003:0E0A       WAVEINGETPOSITION
 0003:0E5A       WAVEINGETID
 0003:0EA4       WAVEOUTGETID
 0003:0EEE       WAVEOUTNOTIFY
 0003:0F06       SOUNDPLAY
 0003:0F30       SOUNDOPEN
 0003:1016       SOUNDCLOSE
 0003:1074       SOUNDWAIT
 0003:108C       SOUNDFREE
 0003:10A6       SOUNDLOADFILE
 0003:11A4       SOUNDLOADMEMORY
 0003:1202       SOUNDINITWAVHDR
 0003:136C       WAVEOMESSAGE
 0003:13D4       WAVEOIDMESSAGE
 0003:1439       WAVEIMESSAGE
 0003:14A1       WAVEIIDMESSAGE
 0004:0000       SNDPLAYSOUND
 0004:0036       DRIVERPROC
 0004:00DC       APPEXIT
 0004:02FE       NEWHANDLE
 0004:0333       FREEHANDLE
 0004:036B       VALIDATEHEADER
 0004:0425       VALIDATEREADPOINTER
 0004:045A       VALIDATEWRITEPOINTER
 0004:0506       VALIDATEDRIVERCALLBACK
 0004:0534       VALIDATECALLBACK
 0004:0563       VALIDATESTRING
 0004:0596       DRVOPEN
 0004:059B       DRVCLOSE
 0004:05A0       DRVGETMODULEHANDLE
 0004:05A5       DRVSENDMESSAGE
 0004:05AA       DRVDEFDRIVERPROC
 0004:05B0       MMTASKYIELD
 0004:05D1       MMGETCURRENTTASK
 0004:05D6       MMTASKBLOCK
 0004:0612       MMTASKCREATE
 0004:06A2       BWINEXEC
 0004:0798       HUGEPAGELOCK
 0004:07C4       HUGEPAGEUNLOCK
 0004:0812       __aFahdiff
 0004:0832       __aFFaulmul
 0004:0832       __aFFalmul
 0004:0854       __aFlmul
 0004:0854       __aFulmul
 0004:0886       __fstrstr
 0005:0000       _mciAppExit
 0005:004B       _szOpen
 0005:0050       MCINOTIFY
 0005:00AA       HANDLENOTIFY
 0005:00E0       MCIBREAK
 0005:0142       MCIAUTOCLOSEDEVICE
 0005:01B0       MCISENDSINGLECOMMAND
 0005:030E       MCISENDCOMMANDINTERNAL
 0005:04E6       MCISENDCOMMAND
 0005:05EE       MCISENDCOMMAND16
 0005:0660       MCICOLONIZEDIGIT
 0005:06F2       MCICOLONIZE
 0005:0778       MCICONVERTRETURNVALUE
 0005:0912       MCISEPARATECOMMANDPARTS
 0005:09FC       MCISENDSYSTEMSTRING
 0005:0AF4       MCIRELAYSYSTEMSTRING
 0005:0BBA       MCIFINDNOTIFY
 0005:0C42       MCIAUTOOPENDEVICE
 0005:0DB0       MCISENDSTRINGINTERNAL
 0005:1386       MCISENDSTRING
 0005:146C       MCIEXECUTE
 0005:155A       MCIGETERRORSTRING
 0005:1626       COULDBE16BITDRV
 0005:1692       IS16BITDRV
 0005:16E2       MCIINITDEVICELIST
 0005:1718       MCIGETDEVICEIDFROMELEMENTID
 0005:17E6       MCIGETDEVICEIDINTERNAL
 0005:188A       MCIGETDEVICEID
 0005:18CE       MCIGETDEVICEIDINTERNALEX
 0005:1906       MCIGETCREATORTASK
 0005:194C       MCIDEVICEMATCH
 0005:19D6       MCILOOKUPTYPE
 0005:1A1C       MCISYSINFO
 0005:1D32       WADDDEVICENODETOLIST
 0005:1DAA       MCIADDDEVICENAME
 0005:1DFA       MCIALLOCATENODE
 0005:1E9C       MCIREPARSEOPEN
 0005:2032       MCIFINDDRIVERNAME
 0005:21E0       MCILOADDEVICE
 0005:259E       MCIEXTRACTDEVICETYPE
 0005:2630       MCIEATTOKEN
 0005:27C6       MCIEXTRACTTYPEFROMID
 0005:284E       MCIOPENDEVICE
 0005:2C76       MCICLOSEDEVICE
 0005:2D1E       MCIGETDRIVERDATA
 0005:2D6E       MCISETDRIVERDATA
 0005:2DC6       MCIDRIVERYIELD
 0005:2E30       MCISETYIELDPROC
 0005:2EAA       MCIGETYIELDPROC
 0005:2F34       MCIBREAKKEYYIELDPROC
 0005:2F8C       MCISETBREAKKEY
 0005:2FA6       MCIEATCOMMANDENTRY
 0005:3022       MCIGETPARAMSIZE
 0005:306A       MCIREGISTERCOMMANDTABLE
 0005:30CA       MCILOADCOMMANDRESOURCE
 0005:32D4       MCILOADTABLETYPE
 0005:3348       MCIFREECOMMANDRESOURCE
 0005:3412       MCIUNLOCKCOMMANDTABLE
 0005:342A       FINDCOMMANDINTABLE
 0005:3518       FINDCOMMANDITEM
 0005:35FA       MCICHECKTOKEN
 0005:3690       MCIPARSEINTEGER
 0005:37F0       MCIPARSECONSTANT
 0005:3886       MCIPARSEARGUMENT
 0005:39F4       MCIPARSEPARAMS
 0005:3D52       MCIPARSECOMMAND
 0005:3DA0       MCIPARSERFREE
 0005:3DF0       MCIMESSAGE
 0005:3E2E       HEAPALLOC
 0005:3E4E       HEAPREALLOC
 0005:3E6F       HEAPFREE
 0005:3E86       DOSCHANGEDIR
 0005:3F06       DOSGETCURRENTDRIVE
 0005:3F0D       DOSSETCURRENTDRIVE
 0005:3F2A       DOSGETCURRENTDIR
 0006:0000       MIDILOCKDATA
 0006:0024       MIDIUNLOCKDATA
 0006:00B4       MIDIOUTGETNUMDEVS
 0006:00D2       MIDIOUTGETDEVCAPS
 0006:011E       MIDIOUTGETVOLUME
 0006:015E       MIDIOUTSETVOLUME
 0006:01C4       MIDIOUTGETERRORTEXT
 0006:0204       MIDIOUTOPEN
 0006:02DE       MIDIOUTCLOSE
 0006:0326       MIDIOUTPREPAREHEADER
 0006:03A4       MIDIOUTUNPREPAREHEADER
 0006:0422       MIDIOUTCACHEPATCHES
 0006:0494       MIDIOUTCACHEDRUMPATCHES
 0006:0506       MIDIINGETNUMDEVS
 0006:0524       MIDIINMESSAGE
 0006:055C       MIDIINGETDEVCAPS
 0006:05A8       MIDIINGETERRORTEXT
 0006:05E8       MIDIINOPEN
 0006:06C2       MIDIINCLOSE
 0006:070A       MIDIINPREPAREHEADER
 0006:0788       MIDIINUNPREPAREHEADER
 0006:0806       MIDIINADDBUFFER
 0006:0870       MIDIINSTART
 0006:08A4       MIDIINSTOP
 0006:08D8       MIDIINRESET
 0006:090C       MIDIINGETID
 0006:0956       MIDIOUTGETID
 0006:09A0       MIDIOIDMESSAGE
 0006:09D7       MIDIIIDMESSAGE
 0007:01E4       MMIORENAME
 0007:02B8       MMIOOPEN
 0007:0454       MMIOCLOSE
 0007:04AE       MMIOREAD
 0007:0624       MMIOWRITE
 0007:07E2       MMIOSEEK
 0007:092A       MMIOGETINFO
 0007:0994       MMIOSETINFO
 0007:0A62       MMIOSETBUFFER
 0007:0CC2       MMIOFLUSH
 0007:0D92       MMIOADVANCE
 0007:0EBA       MMIOSTRINGTOFOURCC
 0007:0F52       MMIOINSTALLIOPROC
 0007:1098       MMIOSENDMESSAGE
 0007:139C       MMIODESCEND
 0007:1590       MMIOASCEND
 0007:16D2       MMIOCREATECHUNK
 0007:17AA       FSTRRCHR
 0007:17DB       MEMCOPY
 0007:17E6       MemCopy386
 0007:182C       MemCopy286
 0008:0000       TIMEGETDEVCAPS
 0008:0022       JOYGETDEVCAPS
 0008:008C       JOYGETNUMDEVS
 0008:00A8       JOYGETPOS
 0008:0112       JOYGETTHRESHOLD
 0008:0176       JOYRELEASECAPTURE
 0008:01DE       JOYSETCAPTURE
 0008:02CE       JOYSETTHRESHOLD
 0008:0318       JOYSETCALIBRATION
 0008:03DE       JOYPOLLCALLBACK
 0008:0572       AUXGETNUMDEVS
 0008:058C       AUXGETDEVCAPS
 0008:05D4       AUXGETVOLUME
 0008:0610       AUXSETVOLUME
 0008:0632       AUXOUTMESSAGE
 0008:0670       JOYMESSAGE
 0008:06A9       NOTIFY_CALLBACK_DATA
 0009:0000       IMIXERMAPID
 0009:0040       IMIXERMESSAGEHANDLE
 0009:006A       IMIXERMESSAGEID
 0009:00C4       MIXERGETNUMDEVS
 0009:00E6       MIXERGETDEVCAPS
 0009:018A       MIXERGETID
 0009:01C6       IMIXERGETID
 0009:0562       MIXEROPEN
 0009:0738       MIXERCLOSE
 0009:07D8       MIXERMESSAGE
 0009:086E       MIXERGETLINEINFO
 0009:0D68       MIXERGETLINECONTROLS
 0009:0EF0       MIXERGETCONTROLDETAILS
 0009:10DC       MIXERSETCONTROLDETAILS
 0009:12DC       INITMIXERTHUNKS
 0009:13A6       MXDMESSAGE
 000A:0000       GWSTACKSIZE
 000A:0002       GWSTACKFRAMES
 000A:0004       GWSTACKUSE
 000A:0006       GWSTACKSELECTOR
 000A:0008       HDRVDESTROY
 000A:000A       VPCALLBACKDATA
 000A:000E       HGLOBAL
 000A:0012       TID32MESSAGE
 000A:0016       MMWOW32LIB
 000B:0006       pLocalHeap
 000B:0006       rsrvptrs
 000B:0008       pAtomTable
 000B:000A       pStackTop
 000B:000C       pStackMin
 000B:000E       pStackBot
 000B:001E       _szJoyKey
 000B:0042       _MCI_wNextDeviceID
 000B:0062       _gIOProcMapHead
 000B:0072       _gpMixerDevHeader
 000B:00E0       _mixerdrv
 000B:00E8       _guTotalMixerDevs
 000B:00EA       _MCI_bDeviceListInitialized
 000B:00EC       _MCI_lpDeviceList
 000B:00F0       CB32
 000B:00F4       WODMAPPER
 000B:00F8       WIDMAPPER
 000B:00FC       _hMciHeap
 000B:00FE       _hwndNotify
 000B:0100       _ghInst
 000B:0102       _pHandleList
 000B:0104       _command_tables
 000B:021C       MCI32MESSAGE
 000B:0220       MOD32MESSAGE
 000B:0224       MID32MESSAGE
 000B:0228       JOY32MESSAGE
 000B:022C       WOD32MESSAGE
 000B:0230       WID32MESSAGE
 000B:0234       _mix32Lib
 000B:0238       AUX32MESSAGE
 000B:023C       _MCI_wDeviceListSize
 000B:023E       _mix32Message
 000B:0242       _lpWavHdr

Program entry point at 0002:0000
